:10000000830100308A009C28F70003088301BF00A9
:100010000408C0000A08C1008A017008C6007108FF
:10002000C7007208C8007308C9007408CA007508C0
:10003000CB007608CC004208C4004308C5008312F8
:1000400003138C1D5C288C118316941A2A288312A2
:10005000A2018316141D382883122108343E84001F
:10006000831300089300A10A0730A10514165B282A
:1000700083121308B300A20A2208023A031D44287F
:1000800033080739A1005B280330220203185128E6
:100090005B28B5172108343E8400831333088000A1
:1000A0005A28210803194928023A03194A28013A13
:1000B00003194A28A10A14138B190B1C812806085E
:1000C0002306F000861F69288E018F010130900001
:1000D0007E2810100230F200F3010F08C300C201A5
:1000E0000E08F000F1014208F0070318F10A430876
:1000F000F107A6277408BC007508BD000608A30018
:100100000B104608F0004708F1004808F2004908C3
:10011000F3004A08F4004B08F5004C08F6004408C8
:10012000C2004508C3004008840041088A003F0817
:100130008300F70E770E0900203084002130B220B2
:10014000213084003430B22083010730C300F53001
:10015000C200343084003F30B6208301C42B040633
:100160008001840A040603190034AF28F000C1207E
:100170008000840A0408700603190034B72883122B
:10018000C200C31BCC28431BD42843088A00420862
:10019000C20A0319C30A8200831343188317420853
:0801A000C20A840000080800F7
:10065000F401F5010310F30CF20C031C362B7008A7
:10066000F40771080318710AF5070310F00DF10D76
:1006700072087304031900342A2B831203138701B1
:10068000EF3083168500FD30860018308700473034
:100690008100043083129200FF30831692000C30E8
:1006A00083129700950183169F010B178B178312F6
:1006B000080083120313A901AA01A90A0319AA0AAF
:1006C00027302A02103003192902031C5D2B05165E
:1006D000A901AA01A90A0319AA0A9C302A024030DA
:1006E00003192902031C6A2B0512592B83120313C9
:1006F000280881000B11BB302402031C852BBE0887
:100700000319832BBE0335158A2B26083E02031CD2
:10071000BE0A351126083E020318902B3E08912B85
:100720002608B200350806390319982B0512992BB3
:100730000516201C9D2B01309E2B0030F000861CDE
:10074000A32B0130A42B0030F0060319B22B15089F
:10075000031DB02B201CAE2B8614C22B8610C22B7F
:100760009503C22B15083206031DBA2B3510A701BD
:10077000A801C22B150832020318C12B95033510AE
:10078000C22B950A830108003D23EA2BB030831663
:1007900093001624B230831693001624B4308316C7
:1007A00093001624B630831693001624B8308316AF
:1007B00093001624BA30831693001624BC30831697
:1007C00093001624BE30831693001624B525D72433
:1007D0009D26142C06083C39F200F301112C7208F6
:1007E0000319C62B043A0319CA2B0C3A0319CE2B52
:1007F000043A0319D22B1C3A0319D62B043A0319D5
:10080000DA2B0C3A0319DE2B043A0319E22B3C3A9B
:100810000319E62B043A0319E72B0C3A0319E82BCA
:10082000142C73080319EF2B59239C2883120313EC
:10083000AA01803083169400363083129400831608
:10084000910183128C1183168C15993083129F00AD
:100850001F150A30BB00071C2F2CE030302C033052
:100860008700B51B5B2C682C2010F3303602031870
:10087000592C3608AB00A6007D30F200F301370892
:10088000F000F1012823E830F4070318F50A0330DB
:10089000F507F409F509F40A0319F50A7408A70025
:1008A0007508A80081000B113514B513682C2014AD
:1008B000352CF3303A2C3408013A0319342C033A1E
:1008C0000319572C2010AB01A60195017E30B50508
:1008D0001F1DCF2CD32C1E08A400B900A1309F00EF
:1008E000071C742CE030752C03308700AA01AA0A7B
:1008F000AC01AD01071C7E2CE0307F2C033087005B
:10090000AC0A0319AD0A2D08803AF000803070025D
:10091000193003192C02031C7A2CCD2C1E08A500BB
:10092000B80099309F00071C972CE030982C0330BA
:100930008700AA01071C9E2CE0309F2C0330870003
:10094000C83025020318CA2C290825060319CD2C06
:100950002508A900B53025020318B02CB530A50034
:100960002B08F200F3012508F000F1014C30F007EC
:100970000318F10AFF30F10728237408F000750806
:10098000F1001430F2000030F301A6277408A6002D
:10099000B514CD2C2B08A600B5101F15D32C2A0892
:1009A00003196B2C8E2C0B1D2B2C76232B2C8312D6
:1009B0000313AB01AC01A701FC30A80081000B11AF
:1009C00099309F001F15071CE72CE030E82C0330FE
:1009D00087001F1DAA2DB12D1E08A40091309F0075
:1009E000071CF42CE030F52C03308700AB01AB0A78
:1009F000AD01AE01071CFE2CE030FF2C0330870058
:100A0000AD0A0319AE0A2E08803AF0008030700259
:100A1000193003192D02031CFA2CA82DF3301E02E5
:100A20000318142D1E08152DF330AC00201487195F
:100A30002010831203132C0829060319242D2C08D7
:100A4000A900A701FC30A800201C282D0130292D69
:100A50000030F000861C2E2D01302F2D0030F006C6
:100A60000319352DA701FC30A800A1309F00071CF9
:100A70003B2DE0303C2D033087000230AB00AD0150
:100A8000AE01071C452DE030462D03308700AD0A2E
:100A90000319AE0A2E08803AF00080307002193037
:100AA00003192D02031C412DA82D1E08A500993005
:100AB0009F00071C5D2DE0305E2D03308700AB01E9
:100AC000071C642DE030652D03308700C8302502F7
:100AD0000318902D2A0825060319932D2508AA002E
:100AE000B53025020318762DB530A5002C08F2008C
:100AF000F3012508F000F1014C30F0070318F10A6A
:100B0000FF30F10728237408F0007508F100143055
:100B1000F2000030F301A6277408A600B514932D47
:100B20002C08A600B510AD01AE01071C992DE030D0
:100B30009A2D03308700AD0A0319AE0A2E08803AB9
:100B4000F00080307002193003192D02031C952D1E
:100B50001F15B12D2B080319EC2C013A03190E2D8A
:100B6000552D0B1DE32C7623E32C83120313AB01CD
:100B7000AC01A701FC30A80081000B1199309F0047
:100B80001F15071CC52DE030C62D033087001F1D23
:100B9000922E992E1E08A40091309F00071CD22D82
:100BA000E030D32D03308700AB01AB0AAD01AE01BD
:100BB000071CDC2DE030DD2D03308700AD0A031962
:100BC000AE0A2E08803AF000803070021930031906
:100BD0002D02031CD82D902E84301E02031CF72DED
:100BE0001E087D3EF0007007AC002010032E7D3003
:100BF0001E020318022E1E087D3CF0007007AC0098
:100C00002014032EAC012C08290603190C2E2C08E5
:100C1000A900A701FC30A800201C102E0130112EC5
:100C20000030F000861C162E0130172E0030F00622
:100C300003191D2EA701FC30A800A1309F00071C3E
:100C4000232EE030242E033087000230AB00AD01AC
:100C5000AE01071C2D2EE0302E2E03308700AD0A8A
:100C60000319AE0A2E08803AF00080307002193065
:100C700003192D02031C292E902E1E08A500993061
:100C80009F00071C452EE030462E03308700AB0145
:100C9000071C4C2EE0304D2E03308700C830250253
:100CA0000318782E2A08250603197B2E2508AA008A
:100CB000B530250203185E2EB530A5002C08F200D1
:100CC000F3012508F000F1014C30F0070318F10A98
:100CD000FF30F10728237408F0007508F100143084
:100CE000F2000030F301A6277408A600B5147B2E8D
:100CF0002C08A600B510AD01AE01071C812EE03016
:100D0000822E03308700AD0A0319AE0A2E08803AFE
:100D1000F00080307002193003192D02031C7D2E63
:100D20001F15992E2B080319CA2D013A0319EC2D12
:100D30003D2E0B1DC12D7623C12D83120313AB0154
:100D4000A701FC30A80081000B110608AA000B10B7
:100D50008B15AA0199309F001F15071CB12EE0309A
:100D6000B22E033087001F1D2D2F312F1E08A40027
:100D7000A1309F00071CBE2EE030BF2E033087003D
:100D8000AA01AA0AAE01AF01071CC82EE030C92E85
:100D900003308700AE0A0319AF0A2F08803AF0002B
:100DA00080307002193003192E02031CC42E2B2F21
:100DB0001E08A50099309F00071CE02EE030E12EB0
:100DC00003308700AA01071CE72EE030E82E03302D
:100DD0008700C83025020318132F29082506031998
:100DE000162F2508A900B53025020318F92EB530B5
:100DF000A5002B08F200F3012508F000F1014C30AA
:100E0000F0070318F10AFF30F10728237408F000F7
:100E10007508F1001430F2000030F301A6277408C1
:100E2000A600B514162F2B08A600B510AE01AF0111
:100E3000071C1C2FE0301D2F03308700AE0A03195A
:100E4000AF0A2F08803AF000803070021930031981
:100E50002E02031C182F1F15312F2A080319B62E36
:100E6000D82E3C08B0003D08B1003D06031D3A2FC6
:100E70003C083006031D312F31082D06031D422F7B
:100E800030082C060319A22FA701FC30A800300857
:100E9000AC003108AD0005303102E03003193002FA
:100EA000031C6C2F08303102343003193002031850
:100EB0006C2F2014073031026D3003193002031CEF
:100EC000652F6C30B0000730B1002130B007031837
:100ED000B10AFA30B107962F05303102D930031923
:100EE00030020318A12F033031028530031930027C
:100EF000031CA12F2010043031024C3003193002A2
:100F00000318862F4C30B0000430B100F001F1011D
:100F10003008F002031CF1033108F102D9307007E8
:100F2000B0000530031806307107B1009C30F200A4
:100F3000F3013108F1003008F00028237508AB00F8
:100F4000A22FAB010B1DAD2E7623AD2EF601F11FA6
:100F5000B02FF009F00A0319F103F1097617F6171B
:100F600073088039F606F31FBC2FF209F20A031941
:100F7000F303F309BC2FF601F401F50172087304C1
:100F8000031DC52FF001F10100341F30F6040310DA
:100F9000F60AF20DF30D031CC82FF30CF20C7308C4
:100FA0007102031DD52F72087002031CDD2F720819
:100FB000F0027308031C730AF102F40DF50DF60B31
:100FC000F61ACD2FF61FE92FF409F40A0319F503D9
:100FD000F5097408F2007508F300761F0034F00973
:100FE000F00A0319F103F10900340034003400342D
:100FF00000340034003400340034DC340534FA3476
:02400E00723FFF
:00000001FF
